:1000000000308A00F92B00007D30840000080319BD
:1000100018280130F800F701F70B0C28F80B0B2813
:100020004A30F700F70B122800000000800B092867
:100030000C2CFD017D08183C031C2F282C307D075B
:100040008316A00045307D07840032308000A20076
:100050002008840022088000FD0A83121A28FF303D
:10006000E200E100EA016A08E900E400E30004308C
:10007000E800E230E7006808E6006708E500F00104
:10008000EF017008EE006F08ED00F4017408F30052
:10009000F200F100EC00EB000130F600F5000F2C4F
:1000A0008316051183120515102CA701A601A501C1
:1000B0000608A4008316851700308312851B0130C3
:1000C000FA000030A4047A08A504122CFE017D0871
:1000D0007E0203188528A3010608A200831685174F
:1000E00000308312851B0130FA000030A2047A0828
:1000F000A30422082406F70023082506FA0077083F
:10010000A6047A08A704FE0A67280034F801F9015A
:10011000F701FA0183162408031D91282308031907
:10012000AB281030A5000310A10DA20DF70DFA0D9C
:1001300024087A02031D9E2823087702031CA7289F
:100140002308F702031CFA032408FA020314F80D2B
:10015000F90DA50B93280000831200341030F7002E
:10016000FA018316A501A20CA10C031CBD282308CB
:10017000FA070318A50A2408A507A50CFA0CF90C20
:10018000F80CF70BB32883120034F701F80183163B
:10019000230803102418F707F70CF80CA418F70726
:1001A000F70CF80C2419F707F70CF80CA419F7074B
:1001B000F70CF80C241AF707F70CF80CA41AF70739
:1001C000F70CF80C241BF707F70CF80CA41BF70727
:1001D000F70CF80C831200348316260828068039A1
:1001E000AA00A61FF828A509A609A50A0319A60AA8
:1001F000A81FFF28A709A809A70A0319A80AF80138
:10020000F901F701FA012808031D09292708031934
:1002100023291030A9000310A50DA60DF70DFA0D26
:1002200028087A02031D162927087702031C1F29B4
:100230002708F702031CFA032808FA020314F80D32
:10024000F90DA90B0B290000AA1F2B29F809F909A0
:10025000F80A0319F90A83120034A901A8015F08FA
:100260007F3C031C6F29831605148312051C462945
:1002700029082B02031C4629031D42292A082802AB
:1002800003184629A80A0319A90A33292B082902A9
:10029000031C5229031D502928082A020318522939
:1002A000DF0A6F29A901A801831605148312051C12
:1002B0005429831605148312051C6229A80A031900
:1002C000A90A59292B082902031C6F29031D6C292F
:1002D00028082A0203186F29DF0AA901A8012C3077
:1002E0005E07840061080002031D8F296308E10096
:1002F000FD017D08183C031C8F292C307D078400EC
:100300006108000203188D295E087D0203198D29FA
:100310002C307D0784000008E100FD0A79292C308B
:100320005E07840063080002031DAE29E301FD019E
:100330007D08183C031CAE292C307D078400000882
:1003400063020318AC295E087D020319AC292C3026
:100350007D0784000008E300FD0A98292C305E0721
:1003600084000008E5020030031C0130E6022C3056
:100370005E078400280880002C305E078400610836
:1003800000020318C8292C305E0784000008E10031
:100390002C305E078400000863020318D4292C3037
:1003A0005E0784000008E3002C305E07840000082C
:1003B000E5070318E60A66088316A200831265089B
:1003C0008316A100A4011930A300831286207808A7
:1003D000E9002C305E078400690800028316A00043
:1003E0002008A01FF5292008003CFE00A008031DDE
:1003F000002A8312EB01F101EE01ED012F2A831691
:10040000A01B032A062AFF30FA00072A01307502D2
:1004100003191B2A01308312EB007E08F100EE0164
:100420007108ED008316A01B162A182AFF30192A1E
:100430000130F500302A8312EB0AEB1B252A6B08EA
:100440007E3C0318252A7E30EB007E0871020318DB
:100450002B2A7E08F1007E08ED070318EE0A8316AA
:1004600083126E088316A20083126D088316A10002
:10047000A401FF30A3008312AE2079088316A200E6
:100480007808A1007108A30083126B088316A400EA
:100490008312C5207808FA01F700F71BFA038316C8
:1004A000A3007A08A4002208A6002108A5002408B9
:1004B000A8002308A7008312EC207808F3001B2C67
:1004C000A901A80160087F3C031CA22A8316851499
:1004D0008312851C792A29082B02031C792A031D03
:1004E000752A2A0828020318792AA80A0319A90AD2
:1004F000662A2B082902031C852A031D832A280843
:100500002A020318852AE00AA22AA901A801831653
:1005100085148312851C872A831685148312851CF3
:10052000952AA80A0319A90A8C2A2B082902031C58
:10053000A22A031D9F2A28082A020318A22AE00AD9
:10054000A901A80145305E07840062080002031D6E
:10055000C22A6408E200FD017D08183C031CC22A7F
:1005600045307D078400620800020318C02A5E0837
:100570007D020319C02A45307D0784000008E2008F
:10058000FD0AAC2A45305E07840064080002031DA2
:10059000E12AE401FD017D08183C031CE12A4530F5
:1005A0007D078400000864020318DF2A5E087D02CC
:1005B0000319DF2A45307D0784000008E400FD0AA6
:1005C000CB2A45305E0784000008E7020030031C98
:1005D0000130E80245305E0784002808800045307D
:1005E0005E078400620800020318FB2A45305E079C
:1005F00084000008E20045305E07840000086402C1
:100600000318072B45305E0784000008E4004530DE
:100610005E0784000008E7070318E80A68088316E5
:10062000A200831267088316A100A4011930A30059
:10063000831286207808EA0045305E0784006A0845
:1006400000028316A0002008A01F282B2008003CD1
:10065000FE00A008031D332B8312EC01F201F00110
:10066000EF01622B8316A01B362B392BFF30FA00CB
:100670003A2B0130760203194E2B01308312EC0025
:100680007E08F200F0017208EF008316A01B492BD0
:100690004B2BFF304C2B0130F600632B8312EC0AFE
:1006A000EC1B582B6C087E3C0318582B7E30EC005A
:1006B0007E08720203185E2B7E08F2007E08EF07A8
:1006C0000318F00A83167008A20083126F088316BD
:1006D000A100A401FF30A3008312AE207908831685
:1006E000A2007808A1007208A30083126C08831688
:1006F000A4008312C5207808FA01F700F71BFA035B
:100700008316A3007A08A4002208A6002108A500E9
:100710002408A8002308A7008312EC207808F4001E
:100720001F2CA101FD017D080F3C031CAF2B031002
:10073000A70CA60C260801398316A00083122708EF
:1007400000398316A100A008031DA92BA1080319D5
:10075000AC2B8312A10A8316FD0A8312932B060881
:10076000A0000310A00C0030861B0130F700770EAC
:100770008316A100A10DA10DC030A1058517003081
:100780008312851B0130F700F70EF70DE030F705F7
:100790007708831621078312A1042A2C831685115A
:1007A000831285110830F800000000000000F817DF
:1007B000EA2BF8138316A00C831203188515031C6B
:1007C00085117817EA2B7813F80BDA2B000000005C
:1007D0000000851584308400840BEC2B0000F81B8E
:1007E000D92B781BE32B00348316051183120511D6
:1007F0008D2C84011F30830507309F0083168511DF
:1008000083128515E0016008DF000130AB00F43091
:10081000AA007830FD000428FF306600192850280F
:10082000DE0155280A30FD006620FC017C08043CEE
:10083000031C292C2D290A30FD006620602A0A306D
:10084000FD006620DE0A5E08193C0319DE01FC0A81
:10085000162C912B75088316A30083126B08831640
:10086000A4008312C5207808FD0076088316A30033
:1008700083126C088316A4008312C5207808FE003A
:10088000FF308316A0008312CE2320088316A00019
:100890008312CE2321088316A0008312CE23690879
:1008A0008316A0008312CE236A088316A000831249
:1008B000CE2361088316A0008312CE23620883161C
:1008C000A0008312CE2363088316A0008312CE23D8
:1008D00064088316A0008312CE2371088316A0003B
:1008E0008312CE2372088316A0008312CE237D08C4
:1008F0008316A0008312CE237E088316A0008312E5
:10090000CE2373088316A0008312CE2374088316A7
:0C091000A0008312CE23112CF42B6300F6
:02400E00193F58
:00000001FF
